:03000000020016E5
:030003000200A850
:100013000200C2D288D28AD2AFC2A8C2AA75F0D9CE
:100023001200741201E474AF1201F774A51201F700
:1000330075400F1201B374A41201F7120102754047
:100043000F1201B37B001200DC75400F1201B37B6A
:10005300081200DC75400F1201B312017175401EC6
:100063001201B374AE1201F775400F1201B302000F
:10007300291201A61201A6C291001201A6D2910073
:100083001201A674A21201F774A01201F774C81228
:1000930001F774291201F71201A674401201F774D3
:1000A300A61201F722C0E0E5F0B4C0030200BF14BA
:1000B300F5F074811201F7E5F01201F7D0E032C0D8
:1000C300E0E5F0B4FF030200D904F5F074811201F6
:1000D300F7E5F01201F7D0E0327AB0EA1201F774D3
:1000E300101201F774001201F779109002217808B9
:1000F300EB9312020CA3D8F8D9F10ABAB8DD227433
:10010300B01201F774101201F774001201F774FFB3
:1001130012020C740112019A74FF12020C74B1FDE5
:100123001201F774101201F774001201F77E0674BE
:10013300FF12020C740012019A74FF12020C0DEDEF
:100143001201F774101201F774001201F7DEE07464
:10015300B71201F774101201F774001201F774FF5C
:1001630012020C748012019A74FF12020C2274B0F2
:10017300FD7F047E02900239ED1201F77410120123
:10018300F774001201F77B8074009312020CA3DB57
:10019300F70DDEE4DFDD227F7EC0E012020CD0E04B
:0F01A300DFF722754032754130D541FDD540F769
:1001B20022D2A8D2AA1201E47541FA75425020A0B7
:1001C2000A1201E4000030A00B80F9D542F0D541BB
:1001D200EAD540E4C2A8C2AA2279197A32DAFED953
:1001E200FA227543047544FA7545C8D545FDD544D0
:1001F200F7D543F122C0E0C290C292C29300F580CB
:1002020000D29400C29400D0E022C0E0C290D29208
:10021200C29300F58000D29400C29400D0E022FF85
:1002220000FF00FF00FF0055AA55AA55AA55AA00D3
:10023200000000000000000404FCFC040404040CA0
:1002420018F0E0000404FCFC0404003078CCC48400
:1002520084083C00000404FCFC0404048CF87000D4
:100262000404FCFC0404000000000000000000C0C4
:10027200300C7CF08000000004040C1C74E480004C
:100282008064140C041C0C040404FCFC0404040C20
:100292001C0404FCFC848484E4041C0000C0F018E8
:1002A200080404040408083C000404FCFC84848060
:1002B2008484FCFC04040020203F3F2020202010E6
:1002C200180F070020203F3F2020003C181020215B
:1002D20021331F0E0020203F3F2121010100000099
:1002E20020203F3F2020202020300C2030382702C1
:1002F200020202233F3C30200000000020203F3F4A
:10030200202000000000000020203F3F20200000AD
:100312000020203F3F2020202320300800070F1814
:1003220030202020202010080020203F3F202000E5
:1003320020203F3F2020001010F0F010101010304D
:1003420060C080001010F0F0101000C0E0301010FB
:100352001020F000001010F0F010101030E0C0007B
:100362001010F0F01010000000000000000000006B
:10037200C030F0C00000000010103070D0900000BB
:1003820000905030107030101010F0F0101010303B
:10039200701010F0F0101010901070000000C0608B
:1003A20020101010102020F0001010F0F01010009B
:1003B2001010F0F01010008080FFFF8080808040DD
:1003C200603F1F008080FFFF808000F061438386D2
:1003D20086CC7C38008080FFFF8484040603010001
:1003E2008080FFFF8080808080C03080C0E09C0BD6
:1003F2000808098FFEF0C080000000008183FEFC27
:1004020082810000000000008080FFFF80800000E9
:10041200008080FFFF8282828F80C020001F3F60A9
:10042200C080808080804020008080FFFF82820226
:070432008282FFFF808000C1
:00000001FF
